:100000000C9462000C94C91A0C94F61A0C948A0091
:100010000C948A000C948A000C948A000C948A0038
:100020000C948A000C948A000C948A000C948A0028
:100030000C948A000C949C0B0C948A000C948A00FB
:100040000C94231B0C948A000C949F1E0C94E21EAB
:100050000C948A000C948A000C948A000C948A00F8
:100060000C94FD080C948A000000000700020100B7
:100070000003040600000000000000000102040864
:100080001020408001020408102001020408102002
:10009000040404040404040402020202020203032E
:1000A00003030303000000002300260029000000D2
:1000B0000000250028002B0000000000240027007D
:1000C0002A00D01F11241FBECFEFD8E0DEBFCDBF66
:1000D00012E0A0E0B1E0E4E1F2E402C005900D928C
:1000E000A23EB107D9F714E0A2EEB2E001C01D9222
:1000F000AC3CB107E1F710E0C4ECD0E004C02297BB
:10010000FE010E94E520C23CD107C9F70E940C20E5
:100110000C9408210C9400008091CE03813019F4D6
:1001200082E08093CE038091CE03833019F484E083
:100130008093CE030895A8950895CF93DF93FC0193
:10014000962F9270862F817060FF20C0992331F026
:100150008091600380831092E20216C0A091E202B7
:10016000C091F903C770D0E0CA56DD4F8881A81747
:1001700010F080E03CC081E08A0F8093E202B0E0A2
:10018000A05FBC4F8C91808381E031C09923C1F086
:1001900090819093E3021092E202292F207E203674
:1001A00051F490916003923020F390819F7190936D
:1001B000A20393E01AC09E3F39F71092600317C064
:1001C0009091E3029F3F01F79091E202993288F605
:1001D00021E0290F2093E2023081E92FF0E0EF5275
:1001E000FC4F3083293281F691E090936003DF91D8
:1001F000CF910895DC01ED91FC910190F081E02D0B
:1002000009950895DC01ED91FC910190F081E02DBC
:10021000099508952091CF033091D003382748E005
:10022000C901880F991F37FF06C09C0151E225279D
:1002300050E1352701C09C01415091F73093D00324
:100240002093CF0308958436910520F4BC0180E00B
:1002500090E017C09C018E3B910528F42A55310986
:10026000AAE0B0E00CC0823D910528F4245B31097E
:10027000A4E6B0E004C02D5C3109A8E5B2E00E941C
:100280001920A4E6B0E09B01AC010E94282008954B
:1002900090E08C599F4F0E942301089581E0809344
:1002A000FA0391E29093FB031092FC038093FD0309
:1002B00082E08093FE0383E08093FF0384E08093D9
:1002C000000485E08093010486E08093020487E0C7
:1002D0008093030486E2809304048093050484E2FF
:1002E0008093060485E280930704089560E08EE021
:1002F0000E94311C61E08FE00E94311C61E080E1CE
:100300000E94311C60E082E00E94311C61E084E0C8
:100310000E94311C089542E050E06CE870E080E0FB
:100320000E94A91A0895E3E0F0E089E08093570065
:10033000E491E67081E0E63009F080E00895CF9323
:10034000DF93C82F0E949301882381F0DFB781E0FB
:100350008093CD03F8940E949B0088E18093600015
:10036000C0936000C1110E949B00DFBFDF91CF915D
:100370000895FC0140A5842F877090E0959587959E
:100380000196242F217030E0820F931F880F880F71
:1003900008958F929F92AF92BF92CF92DF92EF9289
:1003A000FF92CF93FC01C0A5EC2FE770F0E0EA5676
:1003B000FD4FA081B0E0C7FF03C024E130E002C0E0
:1003C0002FE030E0FC0197A183E1989FF001112418
:1003D000E65AFE4F80809180A280B380A20FB31FA7
:1003E00020E43FE14DE750E00E943320A501940155
:1003F0000E946B208C2F887149F469017A01E0ED2D
:10040000CE0EE7E0DE1EE11CF11C1BC0C7FF05C0DD
:1004100060E47AE88CE29EE004C060E07EEE8AEB65
:100420009BE069017A01F8EBCF0EFBE0DF1EE11CD7
:10043000F11CA50194010E946B20C20ED31EE41E84
:10044000F51EC701B60169517C4F8F4F9F4F28EEB3
:1004500033E040E050E00E946B20A8EEB3E00E9441
:100460002820CF91FF90EF90DF90CF90BF90AF907A
:100470009F908F900895DB01FA01582F569590E0D8
:100480002481237030E0322F22274081240F311D38
:1004900011963C932E9344814C70218130E060E4AE
:1004A000469F200D311D112413963C932E931297D5
:1004B00044814073228130E060E1469F200D311D70
:1004C000112415963C932E9314974481407C2381EC
:1004D00030E064E0469F200D311D112417963C93B7
:1004E0002E931697359618969F5F591748F680FFFA
:1004F00047C0408142954695469543702DE431E0D2
:10050000429FC001439F900D11240C9611969C931D
:100510008E93808190E074E0969587957A95E1F7C7
:1005200083709927829FA001839F500D929F500D49
:100530001124445F5F4F13965C934E931297808112
:1005400090E0969587959695879583709927829FD9
:10055000A001839F500D929F500D1124445F5F4F67
:1005600015965C934E93149740814370429FC0014F
:10057000439F900D11240C9617969C938E9316977B
:100580000895803223E0920708F1883E23E0920725
:1005900040F48F519340E4E096958795EA95E1F712
:1005A0000895803D27E0920718F48C5D93400895EC
:1005B000883928E0920768F4885C974074E0969543
:1005C00087957A95E1F78D509C4F089580E090E0F3
:1005D00008958FEF93E008958C30910540F4A4E0E6
:1005E000880F991FAA95E1F7885D9C4F0895843F75
:1005F00023E0920718F484529C4F0895811524E05B
:10060000920740F48657934FF4E0880F991FFA95AC
:10061000E1F7089580E998E008959C0136952795C3
:1006200025753575821B930B9C0123733373969547
:1006300087959695879583739373820F931F9C017B
:1006400054E0369527955A95E1F7280F391F2F70FA
:100650003F7041E051E0249FC001259F900D349FE1
:10066000900D1124892F08954298882319F00000D5
:10067000419A02C0000041980000429A000008958B
:10068000429A000086B14298000081700895CF938D
:10069000DF93D82F5C9A42985C98C8E08D2F8078C1
:1006A0000E943403DD0FC150C9F74298DF91CF910A
:1006B00008958F770E9447030895CF93DF93D82F33
:1006C000C8E08D2F80780E943403DD0FC150C9F738
:1006D0004298DF91CF910895CF93DF934298C8E07D
:1006E00080E0D82FDD0F0E9440038D0FC150C9F765
:1006F000DF91CF9108950E9459030E946C035C9A88
:100700000895A1E0B0E0E7E8F3E00C94BC20806835
:1007100069830E9447036981862F0E945D035C9A6A
:100720002196E2E00C94D820CF93C091DA03C82739
:10073000E82FF0E0EF52FC4F678589E70E948103C4
:100740006C2F8DE30E9481036C2F82E40E94810351
:10075000CF91089586E20E947B030895CF938BE2A8
:100760000E947B03C82F8CE20E947B03282F30E07D
:1007700066E0369527956A95E1F744E0C49FC0018D
:100780001124822B932BCF910895CF93DF93EC010B
:100790006C818CE10E9481036D818DE10E94810357
:1007A0006E818EE10E9481036F8180E20E9481034D
:1007B000688581E20E948103698582E20E9481034B
:1007C0006A8583E20E9481036B8584E20E94810333
:1007D0006C8585E20E9481036D858AE20E94810317
:1007E0006E858EE60E9481036F858FE60E948103ED
:1007F000688980E70E948103698981E70E948103FB
:100800006A8982E70E948103DF91CF910895CF9298
:10081000DF92EF92FF92CF93DF936B017C01C114C3
:1008200088E3D8068CE9E8068CE1F80628F5C701CC
:10083000B60120E836E948E950E00E946B20E90162
:10084000689760E879E687E69FEF0E943B206C0D91
:100850007D1D8E1D9F1DF2E0660F771F881F991F5B
:10086000FA95D1F721E732E040E050E00E946B209A
:10087000F22EE32E80E421C0C701B60120E03DE264
:1008800041E351E00E946B20E901689760E073ED5D
:100890008EEC9EEF0E943B206C0D7D1D8E1D9F1DDA
:1008A000660F771F881F991F21E732E040E050E074
:1008B0000E946B20F22EE32E80E66C2F6F71680F82
:1008C00085E70E9481036E2D86E70E9481036F2DCC
:1008D00087E70E948103DF91CF91FF90EF90DF9037
:1008E000CF9008958F929F92AF92BF92CF92DF9256
:1008F000EF92FF92CF93DF93D82F83E00E947B0388
:100900008093CC0384E00E947B038093CB0360E060
:1009100086E00E94810361E087E00E9481036FE727
:1009200089E00E94810365E08AE00E94810362E120
:100930008BE00E94810365E18CE00E9481036DEFF2
:100940008DE00E94810360E08EE00E948103DD2340
:1009500019F087E491E008C02091F80333E1239F68
:10096000C0011124865A9E4F0E94C5036CE880E3A3
:100970000E9481036FE082E30E94810362E483E3CB
:100980000E9481038091F90387FF02C064E101C0E6
:100990006AE084E30E9481036AE285E30E948103A6
:1009A0006DE286E30E94810364ED87E30E94810388
:1009B00060E088E30E94810360E089E30E94810394
:1009C000D11109C0C090DA03D090DB03E090DC03C2
:1009D000F090DD0307C0C5E9CC2EC1ECDC2EED2C78
:1009E000CEEDFC2ECAE38F2C9924AA24BB24682DBB
:1009F0008C2F0E948103682D85E08C0F0E9481035B
:100A0000FE2CED2CDC2CCC24CF5FCE3361F76FEFC6
:100A100083E40E9481036FEF84E40E9481036FEFFF
:100A200085E40E9481036FEF86E40E948103DD2349
:100A300011F066E002C06091DE038DE60E94810342
:100A400060E089E70E9481036091DF038AE70E94EA
:100A5000810360E083E70E94810360E084E70E94F5
:100A60008103D11109C06091D6037091D7038091A1
:100A7000D8039091D90304C060EC72E98DEE99E13E
:100A80000E940704DF91CF91FF90EF90DF90CF900D
:100A9000BF90AF909F908F90089561E087E00E9493
:100AA000810364E28EE70E94810363E088E00E9494
:100AB000810360E088E00E94810365E087E00E9496
:100AC000810362E085E00E94810383E00E947B0352
:100AD0008093CC0384E00E947B038093CB03089532
:100AE00083E00E947B038093CC0384E00E947B031D
:100AF0008093CB0361E087E00E9481036AE070E0AD
:100B000080E090E00E949C1B0E944D05000008952B
:100B1000CF92DF92FF920F931F93CF93DF931F9299
:100B2000CDB7DEB7082F162F8EE399830E9481037D
:100B3000F02EC02E9981D92E8C2D8F19811738F463
:100B4000F60161916F018FE70E948103F5CF64E0A8
:100B500085E00E94810383E00E947B038093CC03A5
:100B600084E00E947B038093CB030E94791B6093F7
:100B7000C7037093C8038093C9039093CA0369E0C5
:100B800087E00E94810381E08093CE030F90DF9184
:100B9000CF911F910F91FF90DF90CF9008950F9309
:100BA0001F930E9488058091CE03813099F40E94A2
:100BB000791B0091C7031091C8032091C90330919C
:100BC000CA03601B710B820B930B603A764881401D
:100BD000910548F38091CE03813031F46AEB71E0E6
:100BE00082E294E00E943B1D1F910F9108950F93A4
:100BF0001F938091CE03823021F41092CE0381E0C6
:100C000020C08091CE038130D9F40E94791B0091DD
:100C1000C7031091C8032091C9033091CA03601B18
:100C2000710B820B930B613A76488140910540F03D
:100C300061E087E00E9481031092CE0382E001C050
:100C400080E01F910F910895EF92FF920F931F93F1
:100C5000CF93DF938B019C01442737FD4095542FA0
:100C600060E271EA87E090E00E948D20E9011C16A5
:100C70001D0614F0C1E0D0E0D80120E231EA47E0DF
:100C800050E00E9433209E01442737FD4095542FA9
:100C90000E948D20790100E010E00E151F055CF424
:100CA000419ACE010E94C21B4198CE010E94C21BF4
:100CB0000F5F1F4FF2CFCDB7DEB7E6E00C94D42024
:100CC000CF93DF932D9A60910A0470910B04809169
:100CD0000C0490910D040E94070460E089E70E94D3
:100CE000810361E070E080E090E00E949C1B0E9424
:100CF000AA03C82F61E070E080E090E00E949C1B96
:100D00000E94AA03D0E0C80FD11D61E070E080E02E
:100D100090E00E949C1B0E94AA03C80FD11D61E0B5
:100D200070E080E090E00E949C1B0E94AA032D9836
:100D30009E01280F311DC901969587959695879537
:100D4000DF91CF910895CF93C82F2D9A83E00E9411
:100D50007B038093CC0384E00E947B038093CB03CE
:100D600060E086E00E94810361E087E00E948103E9
:100D70006FE789E00E94810365E08AE00E948103B9
:100D800062E18BE00E94810365E18CE00E948103B7
:100D90006DEF8DE00E94810360E08EE00E94810390
:100DA0006CE280E70E94810360E080E30E9481039F
:100DB00060E089E70E94810365E08AE70E94810381
:100DC00062E181E70E94810362E082E70E94810381
:100DD00060E083E70E94810360E084E70E94810372
:100DE00060910A0470910B0480910C0490910D04A1
:100DF0000E94070467E08DE60E9481036AE070E0CC
:100E000080E090E00E949C1B69E087E00E948103E3
:100E10006AE070E080E090E00E949C1BCC2369F0C7
:100E2000C5E1C15009F459C061E070E088EB91E080
:100E30000E9424060E949B00F4CF61E070E088E8E5
:100E400091E00E9424060E949B0065E08DE60E94CE
:100E500081036AE070E080E090E00E949C1B61E00A
:100E600070E088EB91E00E9424060E949B0064E001
:100E70008DE60E9481036AE070E080E090E00E94CD
:100E80009C1B61E070E08DE591E00E9424060E94C9
:100E90009B0062E08DE60E9481036AE070E080E0E2
:100EA00090E00E949C1B61E070E08FEA90E00E945D
:100EB00024060E949B0060E08DE60E9481036AE0A8
:100EC00070E080E090E00E949C1B62E070E085E0B2
:100ED00091E00E9424060E949B0061E087E00E944E
:100EE00081032D98CF910895CF93DF93EC014AE0D1
:100EF00050E06D2F70E082E294E00E94001E6EE2EE
:100F000082E294E00E941F1DBE0184E07695679501
:100F10008A95E1F76F7077274AE050E082E294E02B
:100F20000E94001E6EE282E294E00E941F1DBE013C
:100F30006F7077274AE050E082E294E00E94001E42
:100F4000DF91CF910895D82FC0E0CD1780F4439A58
:100F500064E670E080E090E00E949C1B439864E6A9
:100F600070E080E090E00E949C1BCF5FEECF6CE2CF
:100F700071E080E090E00E949C1BE6CF0F931F93EE
:100F8000CF93DF93EC01062F15E0115051F0CE0105
:100F90000E94F220081741F0602FCE010E94FA2033
:100FA000F4CF82E00E94A307DF91CF911F910F91B0
:100FB0000895A0E0B0E0EFEDF7E00C94AE20482EED
:100FC000562EC0E0D0E0612C712CE12CF12C00E019
:100FD00010E0442079F081E04816A1F092E0491237
:100FE00019C028E4622E712C30E2E32EF12C03E6C6
:100FF00013E010C0612C712C6BE1E62EF12C0AEF8E
:1010000013E008C04DE1642E712C59E2E52EF12C5D
:1010100001ED13E043018C0E9D1E1092D00310923F
:10102000CF033401A62CA818B12CC30101966C0182
:10103000AE14BF04A8F4A00EB11E511006C0C30127
:101040000E94F220F501808305C0F5016081C30193
:101050000E94BE07F50180810E940A013601E2CF9D
:10106000C301511018C0C3010E94F220B82EC6015E
:101070000E94F2202B2D30E0322F2227282B809146
:10108000CF039091D0038217930779F4C0E0D0E0AA
:10109000552453949ECF36016091D0030E94BE0721
:1010A0006091CF03C6010E94BE07D395C13093E083
:1010B000D90708F48ECF852DCDB7DEB7E0E10C94CB
:1010C000CA2060E081E00E94D907882331F081E0E6
:1010D0009091D103983309F080E0089561E081E0B8
:1010E0000E94D907089561E082E00E94D90708951F
:1010F00060E082E00E94D907811108C0E3E6F3E0D6
:101100001192119283E0E338F807D1F70895A1E036
:10111000B0E0EDE8F8E00C94BC2089830E944E0119
:1011200092E0909308049FEF909309049AE09093C3
:101130001204109213041092140410920A041092D4
:101140000B0410920C0410920D042EE120930E0457
:1011500090930F0428EB3BE030931104209310048C
:101160008981882371F061E080E00E94D907E3E67D
:10117000F3E01192119283E0E338F807D1F70E946F
:1011800073082196E2E00C94D82060E080E00E9491
:10119000D907811103C081E00E9487080895CF9389
:1011A000C1E0811101C0C0E06C2F82E10E946A1C85
:1011B0006C2F83E10E946A1C1092C1031092C0033D
:1011C0008091B9008C6F8093B90080E28093B80061
:1011D00085E48093BC00CF91089585ED8093BC0099
:1011E0008091BC0084FDFCCF0895ECEBF0E0108210
:1011F00085E480831092C00308951F920F920FB66A
:101200000F9211242F933F934F935F936F937F938C
:101210008F939F93AF93BF93EF93FF93CF93DF93FE
:101220001F92CDB7DEB78091B900887F803609F470
:10123000C7C0A8F5883209F464C098F4803109F475
:101240005DC038F4882309F4F3C0883009F456C02F
:10125000F1C0883109F455C0803209F0EBC082E05A
:10126000A7C0803409F477C078F4803309F45FC0F4
:10127000883309F0DFC084E08093BF038091C0030E
:101280008B7F8093C003D0C0803509F452C088356D
:1012900009F467C0883409F0CDC085E089C0883979
:1012A00009F4C0C0A8F4883709F48AC038F4883635
:1012B00009F486C0803709F483C0BCC0883809F4BB
:1012C000B1C0803909F47FC0803809F0B3C07BC059
:1012D000803B09F493C038F4803A09F48CC0883A12
:1012E00009F48CC0A7C0803C09F49EC0883C09F476
:1012F0009BC0883B09F09EC080E081C08091C40300
:1013000013C08091C1039FEF980F9093C10388236E
:10131000D1F1E091C203F091C303CF010196909304
:10132000C3038093C20380818093BB007DC083E0B0
:101330003FC0E091C203F091C303CF0101969093A7
:10134000C3038093C2038091BB0080838091C1035B
:1013500081508093C1038091C103823008F064C042
:1013600061C0E091C203F091C303CF010196909355
:10137000C3038093C2038091BB0080838091C1032B
:1013800081508093C1038091C0038B7F8093C00301
:101390008091C00380FF4CC08091C0038E7F8093FA
:1013A000C0038091C00382608093C00384EA3DC083
:1013B0008093BF038091C0038B7F8093C00338C0AC
:1013C0001092C10331C0E091C503F091C60330977C
:1013D00049F18091BB0089838091C10391E0980F0E
:1013E0009093C103811102C062E001C060E0CE01B0
:1013F0000196099515C00E94ED0816C081E0E091A4
:10140000C503F091C603309769F0882311F063E0BB
:1014100001C061E0CE010196099599819093BB00CE
:10142000811102C085E801C085EC8093BC0002C038
:101430000E94ED080F90DF91CF91FF91EF91BF9146
:10144000AF919F918F917F916F915F914F913F915C
:101450002F910F900FBE0F901F9018958F929F9213
:10146000AF92BF92CF92DF92EF92FF92CF93DF9332
:10147000EC010E94791B6B017C014E01A12CB12C67
:101480008091C00382FF11C02097D1F30E94791B85
:101490006C197D098E099F0986169706A806B9065C
:1014A00078F70E94F50881E004C08091BF03109294
:1014B000BF03DF91CF91FF90EF90DF90CF90BF906F
:1014C000AF909F908F900895A2E0B0E0EAE6FAE036
:1014D0000C94B820182F7B01022F047022FD05C048
:1014E00080910B0190910C0102C080E090E02A8372
:1014F00049830E942E0A2A814981811136C01092A7
:10150000BF034093C103F092C303E092C203110FE3
:101510001093C4039091C00321FF02C085E001C075
:1015200084E0892B8093C0038091C00381FF0BC0AE
:101530008091C0038D7F8093C0038091C40380930A
:10154000BB0085EC01C085EE8093BC00822F8170CA
:1015500020FF0BC0011105C080910B0190910C017F
:1015600002C080E090E00E942E0A2296E6E00C94F1
:10157000D420A2E0B0E0EFEBFAE00C94B820182FF2
:101580007B01022F047022FD05C080910B01909118
:101590000C0102C080E090E02A8349830E942E0A59
:1015A0002A814981811138C01092BF034093C10341
:1015B000F092C303E092C203812F880F8160809371
:1015C000C4039091C00321FF02C085E001C084E004
:1015D000892B8093C0038091C00381FF0BC0809151
:1015E000C0038D7F8093C0038091C4038093BB00B0
:1015F00085EC01C085EE8093BC00822F817020FFB6
:101600000BC0011105C080910B0190910C0102C02B
:1016100080E090E00E942E0A2296E6E00C94D4200E
:10162000A0E0B0E0E6E1FBE00C94B6200E94791B5C
:101630000091BB031091BC032091BD033091BE0308
:101640006B017C01C01AD10AE20AF30A97018601F4
:1016500041E1C41647E2D406E104F10408F442C0B3
:101660002091BA0331E0320F3093BA0320FF02C059
:1016700017E001C010E06093BB037093BC0380933C
:10168000BD039093BE0363E070E082E294E00E94A9
:10169000020161E070E082E294E00E94020107E052
:1016A000010F812F90E0EC01CC0FDD1FC35FDE4FF7
:1016B00068817981672F772763707727880F991F53
:1016C000880F991F682B792B82E294E00E94FA0020
:1016D00068817981772782E294E00E94FA001F5F97
:1016E0001013DFCFCDB7DEB7E8E00C94D22025B1E0
:1016F00090E0FC01EE0FFF1FE80FF91FE65DFC4FC5
:101700008081282B25B988B19181892B88B98BB12B
:101710009281892B8BB9089585B1909127038923F4
:1017200085B988B190912803892388B98BB19091AC
:10173000290389238BB908951F920F920FB60F9238
:1017400011242F933F934F935F936F937F938F93C6
:101750009F93AF93BF93CF93EF93FF93C091860373
:1017600080910601C81708F03EC080912503909132
:1017700026039093870080938600EC2FF0E0EE0F15
:10178000FF1FE35FFE4F808191810E94EC02880F72
:10179000991F9093260380932503809125039091B0
:1017A00026032091070130910801281B390B309343
:1017B0000801209307018091100490911104880F73
:1017C000991F2817390720F4909308018093070187
:1017D00080918403811142C08091080480FF41C040
:1017E000C830E0F53EC08091250390912603909388
:1017F0008700809386008091070190910801909363
:1018000026038093250380918403882319F08FEFAA
:101810009FEF06C080912503909126038855924042
:10182000909389008093880080E49CE9909308015C
:101830008093070180918400909185008097D0F378
:101840000E948C0B80918503811105C08091060157
:1018500081500E94770B1092860327C08FEF9FEF75
:1018600006C080912503909126038855924090935D
:1018700089008093880080918400909185008097F2
:10188000D0F30E948C0B80918503811104C080915C
:101890008603811106C0809186038F5F8093860343
:1018A00004C081500E94770BF6CFFF91EF91CF914A
:1018B000BF91AF919F918F917F916F915F914F9168
:1018C0003F912F910F900FBE0F901F90189524E01D
:1018D000829FC00111248C30910538F0853F23E0B0
:1018E000920728F084EF93E008958CE090E008954B
:1018F000CF93DF93C0910904C03390F48C2F807391
:1019000039F0803141F4809187038295807F05C052
:1019100080918C0302C080918D03CF70D0E015C000
:10192000CF33E0F4CF70D0E0809187038295807F41
:101930000E94670CDE01AA0FBB1FA35FBE4F11966A
:101940009C938E93219680918D030E94670CFE01DB
:10195000EE0FFF1FE35FFE4F91838083DF91CF91F6
:10196000089580918803909189039F770E940D03C9
:10197000809387038F3029F480918D03869580585A
:1019800004C099E0899F802D112480938C03F894E2
:101990000E94780C78948091FB038132E1F480916D
:1019A0008C039FEF980F9E3F78F08091B0008F7D61
:1019B0008093B00061E080918C03811101C060E0F0
:1019C00083E00E946A1C08958093B4008091B00067
:1019D00080628093B0000895FF920F931F93CF937E
:1019E000DF930BEF13E0C0E0D0E0B3E0FB2E8C2FD1
:1019F000D801ED918D019E2F907F9031F1F4EF7021
:101A0000F0E0EE0FFF1FE35FFE4F208131816F2D6D
:101A10000E944B20E92FF0E0EE0FFF1FE057FD4F33
:101A200061E0808191818217930708F060E0FE01F8
:101A3000E256FD4F80810E946A1C2196CD30D1056F
:101A4000B1F6CDB7DEB7E5E00C94D5200F931F9328
:101A5000CF93DF9303E613E0C0E0D0E020910904C8
:101A6000822F8F7090E0C817D907E9F00196C81748
:101A7000D90711F42033B8F4F801808191819F7067
:101A8000892B79F0F894F801808191819F700E94F0
:101A9000C102FE01EE0FFF1FE35FFE4F91838083C3
:101AA00078940E94EC0C21960E5F1F4FC031D10537
:101AB000A9F6DF91CF911F910F910895FF920F9397
:101AC0001F93CF93DF9381ED93E00E94B901809340
:101AD000060190910904292F2F70281304C081E07A
:101AE000820F8093060190539F3060F4409106016D
:101AF00030E0842F90E001972817390719F44F5FE1
:101B00004093060180910601813118F080E18093B5
:101B10000601ECE2F3E0DF0112971C92DF0111975E
:101B20001C921082339683E0E335F807A1F74FEF5C
:101B30003FEFADEAB2E00BEF13E02FEFE801899140
:101B40008E018031F8F490E0FD0132976081FC0154
:101B5000EE0FFF1FE80FF91FE65DFC4F8081862B1B
:101B60008083CD010197EC0158818181852B818390
:101B70009C918281892B8283609550959095292331
:101B8000352346231396D4E008301D07B9F6409359
:101B900027033093280320932903CEE9D2E00BEFEB
:101BA00013E0F12CF80181918F01823230F08632FE
:101BB000B8F0863211F460E010C0FBE0FF1204C000
:101BC0008091C1008F7E06C08CE0F81205C0809124
:101BD000C100877F8093C10061E088810E94311C31
:101BE000F3942196EDE0FE12DDCF80910004803267
:101BF00031F461E089E00E946A1C82E801C082E061
:101C00008093800081E0809385038093840380919A
:101C1000FB03813211F08732D9F461E083E00E9446
:101C2000311C60E083E00E946A1C8091FB038132DA
:101C300031F481E08093B0008093B10009C082E06C
:101C40008093B00085E08093B1008EE38093B30071
:101C50008AE1809381008FEF9FEF909389008093BA
:101C6000880080ED97E0909387008093860080E461
:101C70009CE9909308018093070190932603809339
:101C800025031092860380916F00816080936F001E
:101C90008091080483FF0DC08091630390916403D9
:101CA0009F70892B31F00E94260D109284031092B0
:101CB0008503CDB7DEB7E5E00C94D520CF93C82FD0
:101CC000809103048B3221F46C2F8CE00E946A1CFB
:101CD0008091FB03873249F48091B000CC2311F04E
:101CE000806101C08F7E8093B000CF910895A2E201
:101CF000B0E0EDE7FEE00C94AC206B017C010E94AB
:101D00006D1B4B015C0181E00E94720483E08093B3
:101D1000CE030E94700566EC71E082E294E00E94BE
:101D20003B1D7BE1272EE0E53E2EF7E47F2EA6E467
:101D30004A2EB5E55B2EC114D104E104F10469F02B
:101D40000E946D1B681979098A099B096C157D052C
:101D50008E059F0510F080E0D4C08091CE038430C2
:101D600051F764ED71E082E294E00E943B1D8FE741
:101D70000E9459030E946C038AA3823601F501ED8B
:101D800013E00E946C03D8018D938D01B3E00A3FEC
:101D90001B07B9F78091D103883309F0ACC06DED12
:101DA00071E082E294E00E943B1D82E48AA361E03C
:101DB000CE0182960E94CF052D9A81E0A2C0803785
:101DC00041F0893611F581E00E94870889E4898312
:101DD00004C03982C12CD12C76019091CD03809121
:101DE0000804992311F0806801C08F77809308045C
:101DF000EAEFF3E0DE011296822D01900D928A95B2
:101E0000E1F76CE1CE01019674C08437D9F4E4E5C2
:101E1000E98383E08A8381E88B838DE08C838D83E3
:101E20008AE1EDE2F1E0DE01169601900D928A95CD
:101E3000E1F76FE1CE0101960E94CF05C12CD12CB4
:101E4000760159C0853789F40AEF13E00E946C03CC
:101E5000D8018D938D01B4E005311B07B9F761E01E
:101E600080E00E94D9075AA241C08636B9F449825F
:101E7000E3E6F3E0AE014D5F5F4F208131813296A2
:101E8000CA010197DC013C93DA012C934E5F5F4F4E
:101E9000B3E0E338FB0789F761E2B4CF8736C9F4D2
:101EA00003E613E00E946C03682E0E946C03262D4B
:101EB00030E0322F2227280F311DF8012193319372
:101EC0008F01F3E003381F0769F77AA20E947308B5
:101ED0000DC0873481F4E3E6F3E01192119283E0C0
:101EE000E338F807D1F70E9473087AA261E0CE01C7
:101EF00082960E94CF0583E08093CE030E944D0519
:101F00001ACFA296E2E10C94C8201F93CF93DF93DF
:101F1000C82FD62F61E00E94311C61E08C2F0E94F7
:101F20006A1C61E08D2F0E946A1C8AE090E00E948A
:101F3000C21B8D2F0E949D1C892B71F060E08C2F9D
:101F40000E946A1C8AE090E00E94C21B8D2F0E94B2
:101F50009D1C11E0892B09F010E060E08C2F0E949D
:101F6000311C60E08C2F0E946A1C60E08D2F0E9463
:101F70006A1C812FDF91CF911F91089580E4809397
:101F8000BA001092BD008DE990E09093C603809353
:101F9000C5031092600315E004E0C2E0FC2E8091BE
:101FA0006003813039F480E00E947204F092600393
:101FB0004398F5CFC0916003C33061F42D988091B0
:101FC000A2030E949403C093CE030E944D05009388
:101FD0006003E5CF80916003843009F78091CE03E0
:101FE0008430E9F68FE70E945903C0E1D3E0E09125
:101FF000F903E770F0E0EA56FD4F808190E09E0122
:10200000205133402817390724F40E946C03899328
:10201000EECF109360032D9AC2CFAAE2B0E0E3E1C5
:10202000F0E10C94BB201FEF198389E2E1EDF3E0AE
:10203000DE01129601900D928A95E1F721E04AE2C5
:10204000BE016F5F7F4F80E20E94640A81110EC063
:1020500021E041E0BE016F5F7F4F80E20E94B90A3C
:10206000811104C082E08093600302C0109360037A
:1020700080916003823051F00E946D1B60935C037D
:1020800070935D0380935E0390935F03AA96E3E0F1
:102090000C94D720A1E0B0E0E0E5F0E10C94BC2086
:1020A000809160038230D9F48091A203805A8983A1
:1020B00021E041E0BE016F5F7F4F80E20E94640A31
:1020C000882369F08FEF809360030E946D1B6093FB
:1020D0005C0370935D0380935E0390935F0321968E
:1020E000E2E00C94D820A1E0B0E0E9E7F0E10C9444
:1020F000BC20809160038230D1F421E041E0BE0138
:102100006F5F7F4F80E20E94B90A882371F08FEFE2
:10211000809360030E946D1B60935C0370935D036A
:1021200080935E0390935F0302C0898101C08FEFAB
:102130002196E2E00C94D820A2E2B0E0E2EAF0E1DD
:102140000C94AC209E012F5F3F4F80E1D9011D927E
:102150008A95E9F768EE71E082E294E029A33AA358
:102160000E943B1D0E9470051D8A1E8A1F8A188EC0
:10217000312C212C00E0812C912C540180E4482E3C
:1021800081EE582E8DE9682E88E1782E90E5C92ED3
:1021900093ECD92EE12CF12C84EF91E0A0E0B0E09B
:1021A0008D8F9E8FAF8FB8A380EC91EDA8E9BBE136
:1021B000898F9A8FAB8FBC8F80E491EEADE9B8E147
:1021C000898B9A8BAB8BBC8B82E294E00E94071EBA
:1021D000892B09F4E1C082E294E00E94341E9C0144
:1021E00033272C32310509F442C0ACF423323105D7
:1021F00009F0ABC019821A821B821C821D821E82CA
:102200001F82188619861A861B861C861D861E86C6
:102210001F86188A60C02434310529F02335310522
:1022200009F4B2C092C064E482E294E00E941F1DEF
:102230002AE030E040E451EE6DE978E182E294E09A
:102240000E949B1D6CE282E294E00E941F1D2AE026
:1022500030E040EC51ED68E97BE182E294E00E94DD
:102260009B1D6CE282E294E00E944D1DADCF0F5F9A
:10227000043009F0A9CF29813A814B815C81A8EE15
:10228000B3E00E942820698B7A8B8B8B9C8B2D81ED
:102290003E814F8158850E942820698F7A8F8B8FCD
:1022A0009C8F29853A854B855C852D8F3E8F4F8F7E
:1022B00058A32D853E854F8558890E9428206B01A3
:1022C0007C0160323EE473078105910530F462E3DE
:1022D0008CE10E94810300E077CF603345E774070B
:1022E0008105910510F462E2F3CF60345CE9750773
:1022F0008105910510F466E2EBCF80E5C81683EC0A
:10230000D806E104F10410F462E1E2CF90E6C916C8
:102310009AEED906E104F10410F465E1D9CFA0E703
:10232000CA16A1E1DA06A1E0EA06F10410F461E0C0
:10233000CFCFB0EACB16B6E8DB06B1E0EB06F1048E
:1023400010F463E0C5CF65E0C3CF10ED180F1A306D
:1023500008F03ACFE1E0F0E0EC0FFD1F24E0029F2F
:10236000E00DF11D11242081318142815381AAE0C9
:10237000B0E00E942820610F711D811D911D6083B6
:1023800071838283938320CF49885A886B887C88A5
:10239000812C912C540118CF81149104A104B10413
:1023A00089F4C301B2010E94070461E070E080E09B
:1023B00090E00E949C1B1D8A1E8A1F8A188E312C59
:1023C00022242A948D8D9E8DAF8DB8A188169906F2
:1023D000AA06BB06D0F40E94AA032D893E894F8924
:1023E000588D280F311D411D511D2D8B3E8B4F8B5C
:1023F000588F381608F4382E821508F4282E3FEF2F
:10240000831A930AA30AB30A56C0C301B20128EE85
:1024100033E040E050E00E946B20BA01A9012AE0BD
:1024200030E082E294E00E94E91D6CE282E294E0F6
:102430000E941F1D4AE050E0632D82E294E00E945A
:10244000F81D6CE282E294E00E941F1D6D897E8976
:102450008F89988DA50194010E946B20BA01A90172
:102460002AE030E082E294E00E94E91D6CE282E220
:1024700094E00E941F1D4AE050E0622D82E294E049
:102480000E94F81D6CE282E294E00E944D1D4C0C0B
:102490005D1C6E1C7F1C898D9A8DAB8DBC8D841547
:1024A0009505A605B70520F449885A886B887C886D
:1024B000812C912C540129893A894B895C89283EC9
:1024C00033404105510509F07FCEA296E2E10C941C
:1024D000C820A1E0B0E0EFE6F2E10C94BC2080E07F
:1024E0000E949F0161E08DE00E94311C61E081E16A
:1024F0000E94311C0E94760160E080E00E94311C45
:1025000061E081E00E94311C40E052EC61E070E04B
:1025100082E294E00E944F1F0E94C5080E94780842
:1025200065EF71E082E294E00E941C1D81E893E077
:102530000E9474076CE072E082E294E00E941C1D2D
:102540004AE050E063E070E082E294E00E94D11D36
:102550000E948B017894439A67E086E00E94850F81
:10256000882329F043982D980E949C10FBCF65E0AA
:1025700083E00E94850F811104C00E9461088111CF
:1025800019C06FE472E082E294E00E941C1D60E0DA
:1025900070E0CB010E94770E882349F00E946E08FC
:1025A00064E172E082E294E00E943B1D2D9A0E9459
:1025B0005E0D10C00E945E0D80910404823209F00D
:1025C000CAC080910504833209F0C5C08091080417
:1025D00081FDC7C080910404823231F580910504E9
:1025E000833211F581E00E94CF088091080482FFB8
:1025F00008C06FE272E082E294E00E943B1D0E94FC
:10260000BE0F64E170E080E090E00E949C1B21E03E
:1026100041E0BE016F5F7F4F80E20E94B90A8111E5
:1026200003C081E0809360036AE372E082E294E099
:102630000E941C1D8FE00E949F0180E00E94720496
:102640001092A20380E00E94940380E0883170F031
:102650008093E40283E08093CE030E947005809112
:102660006003882371F00E940D100BC021E0280F39
:10267000E82FF0E0EF52FC4F9785992349F3822F22
:10268000E5CF80910704982F9D7F983229F440E090
:1026900052EC61E070E027C0893271F440EA56E8FC
:1026A00061E070E082E294E00E944F1F8091C200DE
:1026B00080628093C2001BC08091F90388718031D1
:1026C00029F440E855E260E070E00DC04091D2038B
:1026D0005091D3036091D4037091D5034A305105D2
:1026E0006105710570F382E294E00E944F1F82E25F
:1026F00094E00E94071E892B29F082E294E00E9458
:10270000341EF5CF80910604843229F08091C100F7
:102710008F7E8093C10080910704853241F08852FA
:10272000833028F08091C100877F8093C100109290
:10273000E6021092E502109262030E94791B6093F8
:102740009E0370939F038093A0039093A10321960F
:10275000E2E00C94D820809108048B7F80930804D9
:1027600035CF82FD37CF64EF71E080E090E00E94CA
:10277000770E882309F42ECF0E946E0864E172E080
:1027800082E294E00E943B1D0E945E0D2D9A22CFB2
:10279000CF93DF9382E294E00E94071E892BE9F039
:1027A000C091E502D0E0CE0101968F71992720916A
:1027B000E60230E08217930781F082E294E00E9403
:1027C000341EC951DD4F88838091E50290E0019667
:1027D0008F7199278093E502DDCFDF91CF91089526
:1027E000A0E0B0E0E6EFF3E10C94B620D82FC62FBE
:1027F0000E94791B0091BB031091BC032091BD0383
:102800003091BE036B017C01C01AD10AE20AF30ABF
:102810009701860141E1C41647E2D406E104F104C0
:1028200008F4D1C16093BB037093BC038093BD03D4
:102830009093BE0380910D0190910E01880F991F16
:102840008093A303892F87702091A403287F282BCE
:102850002093A40380910F0190911001880F991F7C
:10286000382F330F330F330F2770232B2093A403FC
:10287000282F2295269527708091A503807C97703C
:10288000990F990F990F822B892B8093A503209183
:10289000110130911201220F331F922F9295990F3F
:1028A000990F907C8F73892B8093A503932F92951A
:1028B000990F990F907C822F86958695892B80930E
:1028C000A60332FB882780F92091A7032E7F282BAF
:1028D0002093A7038091130190911401880F991FF1
:1028E000382F330F2170232B2093A703382F331F4A
:1028F0003327331F2091A803207F892F8770880FEB
:10290000232B282B2093A803809115019091160169
:10291000880F991F382F3295307F2F70232B2093EB
:10292000A803382F32953F702091A9032078892F72
:1029300087708295807F232B282B2093A903809179
:10294000170190911801880F991F2F772093A903E1
:10295000292F2795222727958695822B8093AA03D6
:10296000892F869583702091AB032C7F282B209391
:10297000AB038091190190911A01880F991F382F8C
:10298000330F330F2370232B2093AB03382F329553
:102990003695369533702091AC03207E892F877051
:1029A000880F880F232B282B2093AC0380911B01C9
:1029B00090911C01880F991F382F3295330F307E6C
:1029C0002F71232B2093AC039295990F907E8695BF
:1029D00086958695892B8093AD0380911D019091FA
:1029E0001E01880F991F8093AE03892F8770209155
:1029F000AF03287F282B2093AF0380911F01909174
:102A00002001880F991F382F330F330F330F277092
:102A1000232B2093AF03282F229526952770809192
:102A2000B003807C9770990F990F990F822B892B97
:102A30008093B0032091210130912201220F331F96
:102A4000922F9295990F990F907C8F73892B809379
:102A5000B003932F9295990F990F907C822F8695B2
:102A60008695892B8093B10332FB882780F92091CA
:102A7000B2032E7F282B2093B203809123019091E3
:102A80002401880F991F382F330F2170232B209397
:102A9000B203382F331F3327331F2091B303207F16
:102AA000892F8770880F232B282B2093B3038091C5
:102AB000250190912601880F991F382F3295307F7C
:102AC0002F70232B2093B303382F32953F70209122
:102AD000B4032078892F87708295807F232B282B41
:102AE0002093B4038091270190912801880F991FAA
:102AF0002F772093B403292F279522272795869592
:102B0000822B8093B503969593708091B6038C7F4A
:102B1000892B8093B6032091290130912A01220F3D
:102B2000331F922F990F990F8370892B8093B603CF
:102B300022952695269523708091B703807E932F4A
:102B40009770990F990F822B892B8093B70320914F
:102B50002B0130912C01220F331F922F9295990F48
:102B6000907E8F71892B8093B703832F8295880F76
:102B7000807E269526952695282B2093B803DD2365
:102B800011F088E001C080E0CC2311F094E001C096
:102B900090E0892B8093B9036FE070E082E294E0CB
:102BA0000E940201C3EAD3E0699182E294E00E94AC
:102BB000611E83E0CA3BD807B9F760E070E082E2AB
:102BC00094E00E940201CDB7DEB7E8E00C94D22079
:102BD000CF93C82F682F82E294E00E94611E8C2F51
:102BE0000E940A01CF910895A0E0B0E0EAEFF5E17C
:102BF0000C94B620C82F0E94791B0091BB03109142
:102C0000BC032091BD033091BE036B017C01C01A4F
:102C1000D10AE20AF30A9701860141E1C41647E2AC
:102C2000D406E104F10408F445C06093BB0370933B
:102C3000BC038093BD039093BE031092D003109207
:102C4000CF0388EA0E94E815CC2311F081E801C087
:102C500081E00E94E81580E10E94E81500E010E0A4
:102C6000F801EE0FFF1FE35FFE4F808191810E940C
:102C7000EC02EC01B3E0CC0FDD1FBA95E1F78D2F2C
:102C80000E94E8158C2F0E94E8150F5F1F4F00313E
:102C9000110531F76091D00370E082E294E00E9468
:102CA000FA006091CF037091D003772782E294E01D
:102CB0000E94FA00CDB7DEB7E8E00C94D220AAE17A
:102CC000B0E0E5E6F6E10C94AE200E949B008CE0BB
:102CD0000E947B0381110BC068E872E082E294E0FD
:102CE0000E943B1D80E00E9472040E9470050E94B9
:102CF000C8130E94791B0E94731091E0853009F07F
:102D000090E01FEF8091CE03843009F4FEC1911151
:102D1000FCC17CC00E94AE0390938B0380938A0316
:102D20002D9AC0929E03D0929F03E092A003F0924E
:102D3000A103109261038091880390918903880F09
:102D4000991F81609093890380938803439880E062
:102D50000E945E0E80911003982F9E7309F02CC282
:102D6000F8948091F90341E153E06DE071E08770E0
:102D70000E943B020E94780C7894909110038091FD
:102D80005A0390FF13C2811124C093E6E92E93E009
:102D9000F92E00E010E0F7018081918194FD0CC0D4
:102DA000F801EE0FFF1FE35FFE4F808191810E94CB
:102DB000EC02D7018D939C930F5F1F4FB2E0EB0E97
:102DC000F11C0031110539F70E94730881E08093EE
:102DD0005A0380916203811103C081E080936203F2
:102DE0001092830310928503109284038091F9035B
:102DF000887109F009C20E94EC0C83E08093CE0335
:102E00000E944D0581E080935B032D980E94791B01
:102E10004B015C010E946D1B6B017C018091610381
:102E2000823008F063C040909E0350909F036090F2
:102E3000A0037090A10380919A0390919B03A091AD
:102E40009C03B0919D0384159505A605B70509F46B
:102E50004DC081ED93E00E94C9016C5D7540810910
:102E6000910995018401041915092609370960178C
:102E7000710782079307D0F540929A0350929B0303
:102E800060929C0370929D030E94AA03282F809356
:102E90008E0380918F0390919003820F911D9093E8
:102EA000900380938F03609191036F5F6093910310
:102EB0006930E0F070E00E945720709390036093B7
:102EC0008F0380918D03E3E08E9F600D711D1124AF
:102ED000769567957695679560938D030E94B10C02
:102EE0001092900310928F031092910380916203CD
:102EF0000091E402882351F110916103101708F04A
:102F000029C240909E0350909F036090A003709050
:102F1000A103A501940124193509460957092F8BEE
:102F2000388F498F5A8F81ED93E00E94C901685113
:102F30007C4F8F4F9F4F2F89388D498D5A8D621747
:102F400073078407950708F4CCC104C280919E03DF
:102F500090919F03A091A003B091A103750164011A
:102F6000C81AD90AEA0AFB0A81ED93E00E94C90156
:102F70009B01AC01A02FB0E00E9428206C157D05BC
:102F80008E059F0558F480929E0390929F03A09215
:102F9000A003B092A10381E080935B03809184033E
:102FA000811116C080910704883219F40E94100B19
:102FB0000FC0893239F460916103809183030E94CC
:102FC000F01306C08A3221F4809183030E94F41525
:102FD00080915B03882309F472C0E091A203EF5F44
:102FE000E093A203E83131F0F0E0EF52FC4F878527
:102FF000811102C01092A20380910A0490910B04E7
:10300000A0910C04B0910D04892B8A2B8B2B09F411
:103010004EC08091920390919303A0919403B0913C
:103020009503892B8A2B8B2B09F441C00E946006E3
:10303000082F10E02091090130910A01369527955B
:10304000369527952C5E3F4F2017310770F40E946C
:103050006D1B68517C4F8F4F9F4F6093920370930D
:1030600093038093940390939503C801880F991F4D
:10307000880F991F4091090150910A019A01220F6E
:10308000331F240F351F820F931F969587959695B2
:10309000879590930A01809309016091D6037091FE
:1030A000D7038091D8039091D9030E94070480919F
:1030B000A2030E9494030E944A1010925B03809125
:1030C00060038F3F09F041C20E946D1B00915C03B9
:1030D00010915D0320915E0330915F03601B710BC3
:1030E000820B930B693E73408105910508F42DC254
:1030F0000E946D1B60935C0370935D0380935E037D
:1031000090935F030E940D1020C20E94791B6B01F7
:103110007C018091CE038430D1F48FE70E94590363
:1031200000E113E0E091F903E770F0E0EA56FD4FAB
:10313000808190E0980120513340281739070CF026
:10314000E9CD0E946C03D8018D938D01EBCFE09106
:10315000F903E770F0E0EA56FD4F40814F5F21E050
:10316000BE016F5F7F4F80E20E94B90A882371F031
:10317000109360030E946D1B60935C0370935D036A
:1031800080935E0390935F0390E0BCCDE091F903E0
:10319000E770F0E0EA56FD4F408150E0BE016E5FFF
:1031A0007F4F80E193E00E94E920BBCD882309F4A2
:1031B00010CE10925A030DCE982F9873983309F0C1
:1031C00008CE90910703892787FF03CE90589093EC
:1031D000070380910704853209F0FBCD10E0212F11
:1031E00030E080911003877090E0821793070CF411
:1031F000F0CD1F5FE12FF0E0E05FFC4F608182E2E5
:1032000094E00E94611EEBCF809107039091100320
:10321000982796FD5AC0807C90E489278093070305
:103220008091E6023091E5028317D1F0E8E0F3E007
:1032300020E02F5F90E0DC01A951BD4F4C914193FC
:1032400001968F719927283011F08313F2CF809364
:10325000E602295C80910703282B2093070335C0E1
:1032600080918E038093080380910404863251F488
:1032700082E10E94C61C95958795959587958093C8
:10328000090302C01092090380910504863251F4AB
:1032900083E10E94C61C95958795959587958093A7
:1032A0000A0302C010920A0380918A0390918B0353
:1032B00090930B0380930C03809188039091890372
:1032C0009F770E940D0380930D0369E087E093E0F0
:1032D0000E9488050E94F70581118DCD0E94C813B8
:1032E000F9CF8091880390918903880F991F90935B
:1032F00089038093880381E080935B03111110C0E0
:10330000C0929603D0929703E0929803F0929903AB
:1033100010929203109293031092940310929503CB
:103320001F5F1093610381ED93E00E94C901640D5A
:10333000751D861D971D60939E0370939F03809358
:10334000A0039093A103439A81E00E945E0E0E9425
:10335000B10C03C0101709F4A7C080916103882342
:1033600009F41CCE809112048823D9F09091830334
:10337000911117C040919603509197036091980363
:103380007091990346015701841A950AA60AB70A53
:1033900090E00E942301681579058A059B0508F4D1
:1033A000B5C0809114048823D9F0909185039111C0
:1033B00017C04091960350919703609198037091C4
:1033C000990346015701841A950AA60AB70A90E0A4
:1033D0000E942301681579058A059B0508F4ADC094
:1033E000809113048823D9F090918403911117C020
:1033F00040919603509197036091980370919903BF
:1034000046015701841A950AA60AB70A90E00E945D
:103410002301681579058A059B0508F492C08091FF
:103420000A0490910B04A0910C04B0910D04892B17
:103430008A2B8B2B09F4B2CD809192039091930348
:10344000A0919403B09195030097A105B10509F4EB
:10345000A5CDC81AD90AEA0AFB0AF7FC9FCD8091CC
:103460000804829581700E94A30680E00E94720485
:103470000E944D050E946D1B6B017C0120910F0481
:1034800030E0A8EEB3E00E941920C60ED71EE81E59
:10349000F91E6894C0F8C0929203D0929303E09210
:1034A0009403F09295037ACD80919E0390919F03AF
:1034B000A091A003B091A10324013501481A590A33
:1034C0006A0A7B0A81ED93E00E94C9019B01AC016D
:1034D000A12FB0E00E942820641575058605970588
:1034E00008F03BCF109289031092880381E080930B
:1034F0005B0310928D030E94B10C80929E03909208
:103500009F03A092A003B092A10327CF81E08093F4
:1035100083030E94260D80910E040E9448016C0DC9
:103520007D1D8E1D9F1D61606093920370939303B8
:10353000809394039093950334CF81E08093850327
:103540004FCF81E0809384036ACF6A96E0E10C94C8
:10355000CA208230E8F4E82FF0E0EE0FFF1FEB5EA8
:10356000FB4F71836083813041F0809169008C7FD3
:10357000842B80936900E89A089580916900440F34
:10358000551F440F551F837F842B80936900E99A50
:1035900008951F920F920FB60F9211242F933F930D
:1035A0004F935F936F937F938F939F93AF93BF934B
:1035B000EF93FF938091150490911604892B29F0C5
:1035C000E0911504F09116040995FF91EF91BF91D8
:1035D000AF919F918F917F916F915F914F913F91AB
:1035E0002F910F900FBE0F901F9018951F920F9262
:1035F0000FB60F9211242F933F934F935F936F93C6
:103600007F938F939F93AF93BF93EF93FF9380919B
:10361000170490911804892B29F0E0911704F09178
:1036200018040995FF91EF91BF91AF919F918F91F0
:103630007F916F915F914F913F912F910F900FBEAE
:103640000F901F9018951F920F920FB60F92112492
:103650002F933F938F939F93AF93BF9380911A04BF
:1036600090911B04A0911C04B0911D043091190489
:1036700023E0230F2D3720F40196A11DB11D05C0B5
:1036800026E8230F0296A11DB11D209319048093F3
:103690001A0490931B04A0931C04B0931D04809102
:1036A0001E0490911F04A0912004B0912104019662
:1036B000A11DB11D80931E0490931F04A0932004AC
:1036C000B0932104BF91AF919F918F913F912F9122
:1036D0000F900FBE0F901F9018952FB7F894609120
:1036E0001A0470911B0480911C0490911D042FBF3B
:1036F00008953FB7F89480911E0490911F04A09103
:103700002004B091210426B5A89B05C02F3F19F0D5
:103710000196A11DB11D3FBF6627782F892F9A2FD3
:10372000620F711D811D911D42E0660F771F881F7A
:10373000991F4A95D1F70895CF92DF92EF92FF92A9
:10374000CF93DF936B017C010E94791BEB01C114C5
:10375000D104E104F10479F00E94791B6C1B7D0B0C
:10376000683E7340A0F381E0C81AD108E108F1086F
:10377000C851DC4FECCFDF91CF91FF90EF90DF90FD
:10378000CF9008950197009739F0880F991F880FFF
:10379000991F02970197F1F70895789484B5826094
:1037A00084BD84B5816084BD85B5826085BD85B5E5
:1037B000816085BDEEE6F0E0808181608083E1E894
:1037C000F0E01082808182608083808181608083CC
:1037D000E0E8F0E0808181608083E1EBF0E08081CF
:1037E00084608083E0EBF0E0808181608083EAE7A1
:1037F000F0E080818460808380818260808380812A
:10380000816080838081806880831092C1000895E8
:10381000833081F028F4813099F08230A1F008954E
:103820008630A9F08730B9F08430D1F480918000DF
:103830008F7D03C0809180008F77809380000895F2
:1038400084B58F7702C084B58F7D84BD0895809143
:10385000B0008F7703C08091B0008F7D8093B0005F
:103860000895CF93DF9390E0FC01E458FF4F24913B
:10387000FC01E057FF4F8491882349F190E0880FC5
:10388000991FFC01E854FF4FA591B49182559F4FB9
:10389000FC01C591D4919FB7611108C0F8948C9137
:1038A000209582238C93888182230AC0623051F450
:1038B000F8948C91322F309583238C938881822BBE
:1038C000888304C0F8948C91822B8C939FBFDF91E6
:1038D000CF910895A1E0B0E0E0E7FCE10C94BA20BC
:1038E000282F30E0F901E859FF4F8491F901E4589D
:1038F000FF4F1491F901E057FF4F04910023C9F0E5
:10390000882321F069830E94081C6981E02FF0E080
:10391000EE0FFF1FE255FF4FA591B4919FB7F894AA
:103920008C91611103C01095812301C0812B8C9370
:103930009FBF2196E4E00C94D620CF93DF93282FED
:1039400030E0F901E859FF4F8491F901E458FF4F45
:10395000D491F901E057FF4FC491CC2391F081112C
:103960000E94081CEC2FF0E0EE0FFF1FEC55FF4FFC
:10397000A591B4912C912D2381E090E021F480E079
:1039800002C080E090E0DF91CF9108958E3008F082
:103990008E5087702091B90190E4299F90011124E5
:1039A000822B80937C0080917A00806480937A00DF
:1039B00080917A0086FDFCCF80917800209179007B
:1039C00090E0922B0895A0E0B0E0E9EEFCE10C94C9
:1039D000B6206C017A01EB01E60EF71E00E010E064
:1039E000CE15DF0561F06991D601ED91FC91019052
:1039F000F081E02DC6010995080F191FF1CFC8010C
:103A0000CDB7DEB7E8E00C94D2206115710589F0DE
:103A1000DB010D900020E9F7AD0141505109461B33
:103A2000570BDC01ED91FC910280F381E02D0995AB
:103A3000089580E090E008950E94051D0895DC013E
:103A4000ED91FC910190F081E02D099508950F937F
:103A50001F93CF93DF93EC016DE00E941F1D8C013B
:103A60006AE0CE010E941F1D800F911FDF91CF9150
:103A70001F910F9108950F931F93CF93DF93EC0144
:103A80000E94051D8C01CE010E94271D800F911FF1
:103A9000DF91CF911F910F9108950F931F93CF93B3
:103AA000DF93EC010E941F1D8C01CE010E94271D97
:103AB000800F911FDF91CF911F910F910895A1E287
:103AC000B0E0E5E6FDE10C94B2207C01C42EE52FC8
:103AD000CB01D22E19A221E02D1510F02AE0D22E12
:103AE0008E010F5D1F4F8D2C912CA12CB12C6C2DB4
:103AF0007E2FA50194010E946B208C2DD29E8019EF
:103B00001124015011098A3010F4805D01C0895CD4
:103B1000F8018083211531054105510521F0C22EA0
:103B2000E32FCA01E4CFB801C7010E94051DA19689
:103B3000ECE00C94CE20A0E0B0E0E1EAFDE10C94D2
:103B4000B620EC016A017B012115310541F4E881C1
:103B5000F9810190F081E02D642F09951DC02A3074
:103B60003105A9F477FF12C06DE20E941F1D8C0180
:103B700044275527BA014C195D096E097F092AE0CF
:103B8000CE010E945F1D800F911F06C02AE0B70181
:103B9000A601CE010E945F1DCDB7DEB7E8E00C9410
:103BA000D2200F931F93CF93DF93EC019A01AB01C7
:103BB000662757FD6095762F0E949B1D8C01CE01D4
:103BC0000E94271D800F911FDF91CF911F910F91B0
:103BD00008952115310549F4DC01ED91FC91019026
:103BE000F081E02D642F099508950E945F1D0895CE
:103BF0009A01462F50E060E070E00E94E91D0895B0
:103C00009A01AB0160E070E00E94E91D0895FC019B
:103C100024853585F901E05CFF4F80819181F901B0
:103C2000EE5BFF4F20813181821B930B8F739927AD
:103C30000895FC0184859585FC01E05CFF4F40817F
:103C40005181FC01EE5BFF4F208131814217530708
:103C500041F00190F081E02DE80FF91F808190E0A4
:103C600008958FEF9FEF0895FC0184859585FC01F1
:103C7000E05CFF4F40815181FC01EE5BFF4F2081F2
:103C800031814217530779F0A081B181A80FB91F84
:103C90008C91208131812F5F3F4F2F7333273183E8
:103CA000208390E008958FEF9FEF0895FC0181A19C
:103CB000882329F0A489B5898C9186FFFBCF11A2B6
:103CC0000895CF93DF93FC0126853785D901A05C49
:103CD000BF4F8D919C91119701968F739927E901A0
:103CE000CE5BDF4F4881598184179507D9F30D903A
:103CF000BC91A02DA20FB31F6C93A685B785A05CC5
:103D0000BF4F11969C938E93A689B7892C9181E021
:103D100090E0078C02C0880F991F0A94E2F7282BC5
:103D20002C9381E081A30488F589E02D8081806453
:103D3000808381E090E0DF91CF91089508951F92F4
:103D40000F920FB60F9211242F933F934F938F939F
:103D50009F93EF93FF938091C00082FD1CC0409120
:103D6000C6008091C8049091C90401968F73992769
:103D70002091CA043091CB048217930771F0E0912F
:103D8000C804F091C904E857FB4F40839093C904DD
:103D90008093C80402C08091C600FF91EF919F916B
:103DA0008F914F913F912F910F900FBE0F901F90C9
:103DB000189582E294E00E94071E892B11F00E9460
:103DC0009E1E08951F920F920FB60F9211242F93EB
:103DD0003F938F939F93EF93FF93209184043091AF
:103DE000850480918604909187042817390731F45F
:103DF0008091C1008F7D8093C10014C0E091860442
:103E0000F0918704EC5BFB4F2081809186049091B8
:103E1000870401968F739927909387048093860473
:103E20002093C600FF91EF919F918F913F912F9129
:103E30000F900FBE0F901F901895A0E0B0E0E3E246
:103E4000FFE10C94B220FC011382128288EE93E011
:103E5000A0E0B0E084839583A683B78386ED92E0EB
:103E6000918380837587648757874687318B208B42
:103E7000138B028BF58AE48AD78AC68AB18EA08E0C
:103E8000938E828E8F85848F8889858F8989868F8E
:103E90008A89878F8B8980A3ECE00C94CE20CF9207
:103EA000DF92EF92FF92CF93DF93EC016A017B01E7
:103EB000411581EE580761057105F9F0EC89FD891E
:103EC00081E090E008A002C0880F991F0A94E2F7F1
:103ED000808360E079E08DE390E0A70196010E9485
:103EE0006B20215031094109510956954795379565
:103EF0002795211580E1380798F0EC89FD8910821B
:103F000060E874E88EE190E0A70196010E946B20C2
:103F10002150310941095109569547953795279503
:103F2000E889F9893083EA89FB89208319A2EE891F
:103F3000FF89408181E090E09C010C8C02C0220F3F
:103F4000331F0A94E2F7422B4083EE89FF894081B8
:103F50009C010D8C02C0220F331F0A94E2F7422B02
:103F60004083EE89FF8940819C010E8C02C0220FA4
:103F7000331F0A94E2F7422B4083EE89FF892081A8
:103F80000F8C02C0880F991F0A94E2F78095822354
:103F90008083DF91CF91FF90EF90DF90CF900895D5
:103FA0008F929F92AF92BF92CF92DF92EF92FF9249
:103FB0000F931F9381E08F9385E08F9387E08F931A
:103FC00083E08F9384E08F93E6EC8E2E912CF2ECBD
:103FD000AF2EB12CA1ECCA2ED12CB0ECEB2EF12CD3
:103FE00004EC10E025EC30E044E454E068E874E0D0
:103FF00082E294E00E941D1F0F900F900F900F908F
:104000000F901F910F91FF90EF90DF90CF90BF9096
:10401000AF909F908F9008950E94CD1B0E946912CF
:10402000C9EDDEE10E945F162097E1F30E94D91EE0
:10403000F9CFA29FB001B39FC001A39F700D811D56
:104040001124911DB29F700D811D1124911D0895A1
:104050000E941920A59F900DB49F900DA49F800DE4
:10406000911D11240895B7FF0C9428200E94282048
:10407000821B930B0895DB018F939F930E9428204E
:10408000BF91AF91A29F800D911DA39F900DB29FF4
:10409000900D11240895991B79E004C0991F96177B
:1040A00008F0961B881F7A95C9F780950895AA1B7A
:1040B000BB1B51E107C0AA1FBB1FA617B70710F013
:1040C000A61BB70B881F991F5A95A9F78095909545
:1040D000BC01CD010895A1E21A2EAA1BBB1BFD0154
:1040E0000DC0AA1FBB1FEE1FFF1FA217B307E407D7
:1040F000F50720F0A21BB30BE40BF50B661F771F2F
:10410000881F991F1A9469F760957095809590950E
:104110009B01AC01BD01CF010895052E97FB1EF454
:1041200000940E94A42057FD07D00E946B2007FC3A
:1041300003D04EF40C94A4205095409530952195D1
:104140003F4F4F4F5F4F08959095809570956195C3
:104150007F4F8F4F9F4F08952F923F924F925F92C4
:104160006F927F928F929F92AF92BF92CF92DF9287
:10417000EF92FF920F931F93CF93DF93CDB7DEB7EC
:10418000CA1BDB0B0FB6F894DEBF0FBECDBF099480
:104190002A88398848885F846E847D848C849B84D7
:1041A000AA84B984C884DF80EE80FD800C811B81E5
:1041B000AA81B981CE0FD11D0FB6F894DEBF0FBE14
:1041C000CDBFED010895EE0FFF1F0590F491E02D96
:1041D0000994FB01DC0102C001900D924150504056
:1041E000D8F70895F999FECF92BD81BDF89A992725
:1041F00080B50895262FF999FECF1FBA92BD81BDD3
:1042000020BD0FB6F894FA9AF99A0FBE0196089558
:04421000F894FFCF50
:104214000000CC04200008409CFF0088130002002A
:10422400020002000200020002000200020002007A
:10423400020002000200020002000200020021004B
:10424400270520082B092209260A230A260B240CF9
:10425400250C280C290C2A8025000005400AA120E1
:104264004EA50020244EA52C2330C01200001A4075
:104274000AA1204EA5001B1E27522C2330802500A6
:104284000005400AA1204EA50020244EA52C233071
:10429400004B000006400AD0009D49007B289D4940
:1042A4002C233000E1000005400A4501D7DC03B8A7
:1042B4001E0EBF00232E48E801008A400A60015503
:1042C4005502AD1E20000023C80154582074696DA6
:1042D400656F7574210057616974696E672062693E
:1042E4006E640A00476F7420706B740A0064617412
:1042F4006120676F6F640A007363616E6E6572207C
:104304006D6F6465004F70656E4C52536E6720523A
:1043140058207374617274696E672000206F6E2078
:104324004857200053617665642062696E64206496
:1043340061746120746F20454550524F4D0A004905
:1043440020616D20736C61766500456E74657269D9
:104354006E67206E6F726D616C206D6F64650045D1
:104364004550524F4D2064617461206E6F74207605
:10437400616C6964206F722062696E64206A756D75
:1043840070706572207365742C20666F7263696E39
:10439400672062696E640A0052582068616E670083
:1043A400B200F4014C0300070B0C101115000305B7
:1043B400060708090A0B0C1213000100000800008C
:1043C4002000004000008001000002000004000002
:1043D4000800001000000010000020000000010090
:1043E400000200000000611EE31C071E341E191E9B
:0243F400561E53
:107E00000F92CDB7DEB7112484B714BE81FFF1D035
:107E100082E08093C00088E18093C10086E0809377
:107E2000C20080E18093C4008EE0CDD088249924E4
:107E3000CC24C394F5E0DF2EE1E1EE2E73E0F72EC3
:107E4000B6D0082F813479F4B2D08983C2D0898129
:107E5000823811F481E005C0813811F485E001C059
:107E600083E09ED09AC0823411F484E103C085344B
:107E700019F485E0B6D091C0853561F498D0082F0B
:107E800010E095D090E0982E8824802A912A880CC2
:107E9000991C82C0863521F484E0A3D080E0E1CF34
:107EA000843609F04CC083D082D0A82E80D0B82E62
:107EB00000E011E07CD0F80181938F01AE16D1F77C
:107EC00088D0FB2DF53489F4E0E0F1E00BC0F9999E
:107ED000FECF92BC81BC0894811C911C819180BD15
:107EE000FA9AF99AEA1598F358C08B2D863409F05E
:107EF00054C0F401F7BEE89507B600FCFDCFF401CD
:107F0000A0E0B1E02C9130E011968C91119790E0B7
:107F1000982F8827822B932B12960C01C7BEE895C9
:107F20001124329681E0A038B80761F7F401D7BE7A
:107F3000E89507B600FCFDCFE7BEE8952EC0843774
:107F4000F1F435D034D0182F32D0B82E42D0FB2DDA
:107F5000F63421F4F40105914F010CC0FB2DF534EA
:107F600049F4F999FECF92BC81BC0894811C911C04
:107F7000F89A00B5802F14D0115049F70EC08537FC
:107F800039F427D08EE10CD085E90AD08FE069CF93
:107F9000813511F488E017D01CD080E101D050CF9A
:107FA0009091C00095FFFCCF8093C600089580910A
:107FB000C00087FFFCCF8091C00084FD01C0A89560
:107FC0008091C6000895E0E6F0E098E19083808318
:107FD0000895EDDF803219F088E0F5DFFFCF84E10E
:107FE000DFCF1F93182FE3DF1150E9F7F2DF1F9166
:0E7FF0000895282E80E0E7DFEE27FF27099492
:027FFE0001057B
:0400000300007E007B
:00000001FF
